:020000040000FA
:02000000802856
:080008008312692069208101C7
:100010000B11A00A0F302002031D54288312860AF8
:10002000A001A10AC730DE20303021076E20EA206F
:100030000A302102031D5428A101A20AC630DE2085
:10004000303022077720EA2006302202031D542890
:10005000A201A30AC430DE20303023076E20EA203C
:100060000A302302031D5428A301A40AC330DE2052
:10007000303024077720EA2006302402031D54285C
:10008000A401A50AC130DE20303025076E20EA2009
:100090000A302502031D5428A501A60AC030DE201F
:1000A00030302607EA2054288B160900A001A10150
:1000B000A201A301A401A501A601080004302502A4
:1000C000031D9E2802302602031D9E285620AD20C7
:1000D0000800BB30A800A80B6B280800A7003A3026
:1000E0002702031D75283030080027080800A700E4
:1000F00036302702031D7E2830300800270808000C
:10010000831600308600850083123830DE200130EF
:10011000DE200330DE200F30DE208030DE20C030D5
:10012000DE20A020AD200730831681008312051049
:100130008601003081008B178B1686015E209E2879
:100140000030A1000030A2000030A3000230A40063
:100150000530A5000130A6000800C730DE20303091
:100160002107EA20C630DE2030302207EA20C530E1
:10017000DE203A30EA20C430DE2030302307EA2087
:10018000C330DE2030302407EA20C230DE203A308F
:10019000EA20C130DE2030302507EA20C030DE20E2
:1001A00030302607EA208030DE205430EA20493003
:1001B000EA204D30EA204530EA2008008600F6208B
:1001C00004308500F62000308500F62004308500DC
:1001D000F62008008600F62006308500F620023062
:1001E0008500F62006308500F62008001930AA00A8
:1001F000A900A90BF928AA0BF8280800FA30AA00D0
:10020000A900A90B0129AA0B00290800FE20FE2045
:02021000FE20CE
:02400E00F13F80
:00000001FF
